:020000040000FA
:100000000C94F2040C941A050C941A050C941A051D
:100010000C941A050C941A050C941A050C941A05E4
:100020000C941A050C941A050C941A050C941A05D4
:100030000C941A050C941A050C941A050C941A05C4
:100040000C94041E0C941A050C94741E0C944E1EF1
:100050000C941A050C941A050C941A050C941A05A4
:100060000C94A61E0C941A0500407A10F35A00A0B6
:10007000724E18090010A5D4E80000E87648170071
:1000800000E40B54020000CA9A3B000000E1F505B1
:10009000000080969800000040420F000000A086FB
:1000A00001000000102700000000E803000000002D
:1000B0006400000000000A000000000001000000D1
:1000C00000002C76D888DC674F0823DFC1DFAE59EB
:1000D000E1B1B796E5E3E453C63AE651997696E87E
:1000E000E6C28426EB898C9B62ED407C6FFCEFBC02
:1000F0009C9F40F2BAA56FA5F490055A2AF75C932D
:100100006B6CF9676DC11BFCE0E40D47FEF520E662
:10011000B500D0ED902E0300943577050080841E45
:10012000080000204E0A000000C80C333333330FA0
:10013000986E12831141EF8D2114893BE65516CF3D
:10014000FEE6DB18D1844B381BF77C1D901DA4BB49
:10015000E424203284725E228100C9F124ECA1E5FE
:100160003D270000000000000000050000000A001C
:1001700000000F00000014000000190000001E0025
:10018000000023000000280000002D0000003200C5
:100190000000370000003C00000041000000460065
:1001A00000004B00000050000000550000005A0005
:1001B00000005F00000064000000ECFFFFFF274824
:1001C0000E00D7571200319D1600F5191B00EBCF1A
:1001D0001F00DEC02400A1EE29000D5B2F000208E5
:1001E000350063F73A00202B410028A547007567CA
:1001F0004E0006745500DCCC5C0005746400926B04
:100200006C0098B5740036547D008F498600CA97FB
:100210008F00F1FFFFFF87C80A0067C40E00ECF4EF
:100220001200CC5B1700C6FA1B009FD320001FE80A
:100230002500163A2B005ACB3000C89D360044B337
:100240003C00B40D430008AF49003599500035CE4D
:10025000570009505F00B72067004F426F00E0B6BB
:100260007700858080005CA18900F6FFFFFFDC3B02
:100270000700EB230B009B3F0F009790130097188C
:10028000180054D91C0091D42100130C2700A88118
:100290002C00223732005C2E380034693E008FE992
:1002A000440059B14B0082C25200011F5A00D2C80B
:1002B0006100FAC169007E0C720070AA7A00E29DAA
:1002C0008300FBFFFFFF46A30300857707005F7EE7
:1002D0000B0077B90F007D2A14001FD3180018B542
:1002E0001D0025D222000A2C280091C42D00899DD2
:1002F0003300CAB839002C18400092BD4600E4AA69
:100300004D000DE2540001655C00BA3564003356BF
:100310006C0070C874007D8E7D000000000000003D
:10032000000070C0030073B20700A9D70B00B23100
:1003300010003BC21400EF8A1900878D1E00BDCB50
:1003400023005047290008022F00AFFD3400193C5C
:100350003B001CBF4100968848006B9A4F0082F614
:100360005600C99E5E0036956600C0DB6E0068745C
:100370007700050000006053FCFF00000000EB6206
:1003800000007FEC07008E2F0C00FCA710006E57BA
:100390001500903F1A0016621F00B5C024002B5DA7
:1003A0002A003A393000AB5636004BB73C00EF5CC0
:1003B00043006F494A00A87E510080FE5800E0CA01
:1003C0006000B8E56800FA5071000A000000D89E8D
:1003D000F8FFA737FCFF000000006DF9030082253D
:1003E0000800D4850C00031C1100B1E9150086F04B
:1003F0001A003232200066B02500DD6C2B005669F1
:10040000310093A737005F293E0089F04400E5FEE4
:100410004B004E565300A2F85A00C5E76200A325D0
:100420006B000F000000F3E3F4FFF468F8FF771CA3
:10043000FCFF0000000019150400515D08003DDAC2
:100440000C00768D11009C781600529D1B0046FD15
:100450002000249A2600A4752C007F91320073EFAF
:10046000380049913F00C7784600C0A74D000720DB
:10047000550078E35C00F0F36400140000005F2492
:10048000F1FF9095F4FF3C34F8FFE201FCFF00001F
:1004900000001E300400C5930800892C0D00FFFBEE
:1004A0001100C303170075451C00BBC22100427D2B
:1004B0002700B9762D00D7B03300572D3A00F9ED5B
:1004C000400081F44700BD424F007ADA56008DBDEE
:1004D0005E0019000000E061EDFF41BFF0FF194927
:1004E000F4FFDA00F8FFFDE7FBFF00000000654ABB
:1004F0000400B4C808007A7C0D0049671200BA8A6B
:10050000170068E81C00F68122000B592800526F82
:100510002E007CC6340040603B005A3E4200886298
:10052000490092CE5000418458001E0000005E9E9B
:10053000E9FFEEE7ECFFF15CF0FFCEFEF3FFF7CE54
:10054000F7FFDECEFBFF00000000DA630400F0FBE3
:100550000800CCC90D00FBCE1200120D1800A785B3
:100560001D00583A2300C82C29009D5E2F0083D11E
:1005700035002E873C0050814300A6C14A00F04957
:10058000520023000000DCDBE5FF9D11E9FFC9718B
:10059000ECFFC2FDEFFFF0B6F3FFBD9EF7FF9BB689
:1005A000FBFF00000000667C04004F2D09003C1496
:1005B0000E00BA321300578A1800A51C1E003EEB2D
:1005C0002300BDF72900C843300001D1360017A130
:1005D0003D00BAB544009F104C00280000007C1C70
:1005E000E2FF6D3EE5FFC489E8FFD9FFEBFF0DA2F6
:1005F000EFFFBF71F3FF5A70F7FF499FFBFF000049
:100600000000F4930400A05C0900875B0E002A92AE
:10061000130015021900D7AC1E00019424002EB956
:100620002A00F81D310002C43700F1AC3E0071DA37
:1006300045002D0000008362DEFFA570E1FF25A7C5
:10064000E4FF5807E8FF8F92EBFF274AEFFF7E2F6A
:10065000F3FFF943F7FF0089FBFF000000006CAADD
:100660000400B9890900649F0E00ECEC1300D673F6
:100670001900AC351F00FB33250055702B0053ECDF
:1006800031008FA93800A9A93F003200000054B002
:10069000DAFFA6AADDFF52CCE0FF9F16E4FFDB8A5B
:1006A000E7FF592AEBFF6DF6EEFF73F0F2FFCA1970
:1006B000F7FFD673FBFF00000000B5BF040067B46E
:1006C00009008DDF0E009F42140020DF190091B653
:1006D0001F007DCA25006D1C2C00F6AD3200AB80DA
:1006E0003900370000007308D7FFF5EED9FFCBFBC8
:1006F000DCFF3530E0FF778DE3FFDA14E7FFAAC7B0
:10070000EAFF3BA7EEFFE2B4F2FFFAF1F6FFE35F88
:10071000FBFF00000000B9D304007BDC0900B71B1D
:100720000F00E392140077431A00F22E2000D756F0
:100730002600ACBC2C00FC6133003C000000876D3F
:10074000D3FF3A40D6FF3938D9FFC056DCFF069DAB
:10075000DFFF4F0CE3FFDBA5E6FFF76AEAFFEE5C85
:10076000EEFF137DF2FFBBCCF6FF3F4DFBFF000019
:1007700000005FE60400C4010A009A530F0051DD37
:1007800014005CA01A00359E200057D82600425065
:100790002D004100000059E2CFFF3BA1D2FF66844B
:1007A000D5FF078DD8FF54BCDBFF8013DFFFCA9352
:1007B000E2FF713EE6FFB914EAFFEA17EEFF4F4988
:1007C000F2FF3CAAF6FF043CFBFF000000008EF79E
:1007D00004000E240A00E8860F008421150050F55D
:1007E0001A00BE032100454E270046000000D269D2
:1007F000CCFFE514CFFF3AE3D1FFF8D5D4FF49EEA3
:10080000D7FF5B2DDBFF6294DEFF9424E2FF2BDF3A
:10081000E5FF68C5E9FF8DD8EDFFE119F2FFB08A69
:10082000F6FF492CFBFF000000002B0705002843C2
:100830000A0054B50F00145F1500CE411B00F05E96
:1008400021004B0000000307C9FF469ECBFFC6579F
:10085000CEFF9F34D1FFF535D4FFED5CD7FFB1AAB1
:10086000DAFF6E20DEFF55BFE1FF9E88E5FF827D47
:10087000E9FF3D9FEDFF14EFF1FF4A6EF6FF2A1EE0
:10088000FBFF000000001F150500DC5E0A008EDE85
:100890000F009695150053851B00500000001EBDEB
:1008A000C5FF9140C8FF3CE5CAFF32ACCDFF8C9636
:1008B000D0FF6AA5D3FFEAD9D6FF3135DAFF69B890
:1008C000DDFFBE64E1FF613BE5FF843DE9FF626C53
:1008D000EDFF35C9F1FF3D55F6FFBF11FBFF0000ED
:1008E00000004D210500F4760A00480210009FC464
:1008F0001500550000007B8FC2FF1FFFC4FFF38E61
:10090000C7FF0540CAFF6513CDFF270AD0FF642546
:10091000D3FF3766D6FFBFCDD9FF205DDDFF811540
:10092000E1FF0DF8E4FFF205E9FF6140EDFF93A858
:10093000F1FFBF3FF6FF2307FBFF000000009B2BEA
:1009400005003B8B0A002D201000CDCCCC3D0AD7F2
:10095000233C17B7D13877CC2B329595E6241FB1BD
:100960004F0A0000803FCDCCCC3D6F12833A95BF3B
:10097000D6337D1D9026B3CE010C0000204100002F
:10098000C84200401C4620BCBE4CCA1B0E5AAEC515
:100990009D7400000008000201000003040700002D
:1009A00000000000000000000000250028002B00CF
:1009B00000000000240027002A00040404040404AA
:1009C00004040202020202020303030303030102FE
:1009D00004081020408001020408102001020408CD
:1009E0001020C51F11241FBECFEFD8E0DEBFCDBF42
:1009F00024E0AAE5B2E001C01D92AD36B207E1F7EE
:100A000012E0A0E0B1E0ECE7F7E502C005900D923E
:100A1000AA35B107D9F714E0C2EFD4E004C021979A
:100A2000FE010E94BB29C13FD107C9F70E9448209F
:100A30000C94BC2B0C94000091E090930D038093D8
:100A40002F0310920E031092300308950895089515
:100A500090E0FC01E253F64F24918654964FFC013E
:100A60008491882399F090E0880F991FFC01E0554C
:100A7000F64FA591B491FC01EA55F64F85919491FA
:100A80008FB7F894EC91E22BEC938FBF089590917F
:100A9000E0028091DF022FEF3FEF981748F4E92F33
:100AA000F0E0E554FD4F208130E09F5F9093E0023D
:100AB000C90108959091E0028091DF022FEF3FEF8E
:100AC000981748F4E92FF0E0E554FD4F208130E01D
:100AD0009F5F9093E002C90108950F931F93CF93F6
:100AE000DF93FC01C081D18117861686CE019F70ED
:100AF0009183808390E080E030E020E0DC01AE7FF5
:100B0000AE0FBF1F5C9111964C9180FF1FC025272F
:100B100048E0D901220F331FB7FF02C050E3352749
:100B20004150B9F701968031910541F7D183C083D7
:100B3000232F332722952F7081E06217130609F0C7
:100B400080E0DF91CF911F910F91089510E024274D
:100B50003127DECF90E0FC01EE56F64F2491FC01E8
:100B6000E253F64F3491FC01E654F64FE491EE2344
:100B7000C9F0222339F0233001F1A8F4213019F112
:100B8000223029F1F0E0EE0FFF1FEA55F64FA59154
:100B9000B4918FB7F894EC91611126C030953E2343
:100BA0003C938FBF08952730A9F02830C9F0243036
:100BB00049F7809180008F7D03C0809180008F77FE
:100BC00080938000DFCF84B58F7784BDDBCF84B581
:100BD0008F7DFBCF8091B0008F778093B000D2CF14
:100BE0008091B0008F7DF9CF3E2BDACF3FB7F894DC
:100BF0008091B7029091B802A091B902B091BA0267
:100C000026B5A89B05C02F3F19F00196A11DB11D67
:100C10003FBFBA2FA92F982F8827BC01CD01620FA3
:100C2000711D811D911D42E0660F771F881F991F5E
:100C30004A95D1F708958F929F92AF92BF92CF922B
:100C4000DF92EF92FF926B017C010E94F6054B014F
:100C50005C01C114D104E104F104B9F00E94F6056D
:100C6000681979098A099B09683E734081059105D5
:100C700080F321E0C21AD108E108F10888EE880E5D
:100C800083E0981EA11CB11CE4CFFF90EF90DF9091
:100C9000CF90BF90AF909F908F900895CF93DF93A8
:100CA000EC0189E00E9428058AE00E9428058BE07B
:100CB0000E942805C330D105A1F160F42297E9F024
:100CC00060E089E00E94AA0560E08AE00E94AA052F
:100CD00060E01CC0C430D10551F1259789F761E06F
:100CE00089E00E94AA0561E08AE00E94AA0561E00D
:100CF0008BE0DF91CF910C94AA0560E089E00E941F
:100D0000AA0560E08AE00E94AA0561E08BE00E94EB
:100D1000AA0565E070E080E090E0DF91CF910C944F
:100D20001B0660E089E00E94AA0561E0CECF60E08A
:100D300089E00E94AA0561E0E5CFAF92BF92CF9211
:100D4000DF92EF92FF920F931F93CF93DF936C018B
:100D50007B018B01040F151FEB015E01AE18BF086C
:100D6000C017D10759F06991D601ED91FC9101901E
:100D7000F081E02DC6010995892B79F7C501DF9136
:100D8000CF911F910F91FF90EF90DF90CF90BF9088
:100D9000AF900895FC0144815581608171818DE59A
:100DA00094E00C949D06FC01538D448D252F30E07A
:100DB000842F90E0821B930B541710F0CF96089568
:100DC00001970895FC01918D828D981761F0A28D95
:100DD000AE0FBF2FB11D5D968C91928D9F5F9F735B
:100DE000928F90E008958FEF9FEF0895FC01918D11
:100DF000828D981731F0828DE80FF11D858D90E07E
:100E000008958FEF9FEF0895FC01918D228D892F1A
:100E100090E0805C9F4F821B91098F739927089502
:100E200081E393E00E94040721E0892B09F420E08C
:100E3000822F089580E090E0892B29F00E9410070E
:100E400081110C9400000895FC01A48DA80FB92F06
:100E5000B11DA35ABF4F2C91848D90E001968F73E2
:100E60009927848FA689B7892C93A089B1898C9101
:100E7000837080648C93938D848D981306C0028850
:100E8000F389E02D80818F7D80830895EF92FF921A
:100E90000F931F93CF93DF93EC0181E0888F9B8D9D
:100EA0008C8D98131AC0E889F989808185FF15C057
:100EB0009FB7F894EE89FF896083E889F98980817A
:100EC0008370806480839FBF81E090E0DF91CF9149
:100ED0001F910F91FF90EF900895F62E0B8D10E06B
:100EE0000F5F1F4F0F731127E02E8C8D8E110CC0DA
:100EF0000FB607FCFACFE889F989808185FFF5CF25
:100F0000CE010E942407F1CFEB8DEC0FFD2FF11DD8
:100F1000E35AFF4FF0829FB7F8940B8FEA89FB8961
:100F200080818062CFCFCF93DF93EC01888D8823BF
:100F3000B9F0AA89BB89E889F9898C9185FD03C03C
:100F4000808186FD0DC00FB607FCF7CF8C9185FF21
:100F5000F2CF808185FFEDCFCE010E942407E9CF3B
:100F6000DF91CF910895089520918B02260F3327AA
:100F7000331F21323105ECF420910703FC0190E08E
:100F800080E0243069F082E00895A0918B022191E5
:100F9000AC0145595D4FA40FB52FB11D2C9301969F
:100FA000861798F380918B02680F60938B0280E024
:100FB000089581E008951092070381E0809306036D
:100FC0001092E10261E082E10E94AA0561E083E102
:100FD0000E94AA05E9EBF0E080818E7F808380810A
:100FE0008D7F808388E48093B80085E48093BC0083
:100FF00008951092E0021092DF0210920E031092F8
:1010000030030E94DB0786E295E09093DE02809336
:10101000DD0287E295E09093DC028093DB02089585
:10102000CF93DF9391E090936A028823B9F0C09147
:10103000B800D091BA008091BC008A7B8093BC003C
:1010400060E082E10E94AA0560E083E10E94AA05B7
:101050000E94DB07D093BA00C093B800DF91CF9114
:101060000895CF92DF92EF92FF920F931F93CF9349
:10107000DF93D091300381E0D13208F09CC0C09161
:101080002F030E94F6056B017C01809107038111FB
:101090006CC082E08093070381E0809306038FEFAA
:1010A0008093050310920403D0930303AFE0B3E0F1
:1010B000E3EEF2E080E0D8138DC01092E20280915E
:1010C000E202CC0FC82BC093E2028091E102813092
:1010D00009F084C01092E1020E94F6056B017C01C8
:1010E0008091E2028093BB008091090390910A03F2
:1010F000A0910B03B0910C03892B8A2B8B2BA1F0B1
:101100000E94F6050091090310910A0320910B0338
:1011100030910C036C197D098E099F09061717077A
:101120002807390708F442C08091BC0083FDD8CF5E
:1011300085EC8093BC000E94F6056B017C018091D8
:101140000703823009F44CC0809105038F3F09F4F6
:1011500069C080910503803209F466C0809105035F
:10116000803309F463C084E026C080910903909124
:101170000A03A0910B03B0910C03892B8A2B8B2BB4
:1011800009F483CF0E94F6050091090310910A0328
:1011900020910B0330910C036C197D098E099F0976
:1011A000061717072807390708F06FCF8091080343
:1011B0000E94100885E010920E03109230031092E6
:1011C0000D03DF91CF911F910F91FF90EF90DF9072
:1011D000CF9008959D9191938F5F6DCF85EEA9CFAC
:1011E0008091090390910A03A0910B03B0910C0325
:1011F000892B8A2B8B2B09F4A2CF0E94F605009134
:10120000090310910A0320910B0330910C036C1910
:101210007D098E099F09061717072807390708F067
:101220008ECFC4CF80E0C7CF82E0C5CF83E0C3CFED
:101230000895E091E0028091DF02E81730F4F0E0D9
:10124000E554FD4F808190E008958FEF9FEF089562
:101250008091DF029091E002891B990B0895CF9253
:10126000DF92EF92FF920F931F93CF93DF937C0156
:10127000CB018A0120910D03222389F0EB016B0140
:10128000C40ED51ECC15DD0569F06991D701ED912D
:10129000FC910190F081E02DC7010995F3CF642FF7
:1012A0000E94B407C801DF91CF911F910F91FF9069
:1012B000EF90DF90CF900895CF93DF931F92CDB73B
:1012C000DEB7698320910D032223F9F020913003CA
:1012D000203258F021E030E0FC013383228390E09B
:1012E00080E00F90DF91CF91089580910E03E82F59
:1012F000F0E0E15FFC4F998190838F5F80930E0354
:101300008093300381E090E0ECCF61E0CE01019664
:101310000E94B407F7CF0F931F93CF938C01C62F72
:10132000FC0184810E941C05F80163856C2B8EEC06
:1013300093E00E945C09CF911F910F910C943108AA
:1013400090E080E00895CF93DF93EC01888199814C
:10135000DC01ED91FC910190F081E02D09952A814D
:101360003B81820F931F9B838A83DF91CF910895E6
:10137000CF93DF93EC0188819981DC01ED91FC91A1
:101380000280F381E02D09952A813B81820F931F12
:101390009B838A83DF91CF9108958F929F92AF9222
:1013A000BF92CF92DF92EF92FF920F931F93CF9352
:1013B000DF93CDB7DEB766970FB6F894DEBF0FBEEA
:1013C000CDBF6C018E01095E1F4F78018AE0882E27
:1013D000912CA12CB12CCB01BA01A50194010E9442
:1013E0001F28942F852F605DF80162938F01A9015A
:1013F000692F782F411551056105710561F7A70126
:101400004E1B5F0BBF01C6010E94B80966960FB65E
:10141000F894DEBF0FBECDBFDF91CF911F910F912A
:10142000FF90EF90DF90CF90BF90AF909F908F9004
:101430000895FC012581222339F0F8E02F02900164
:101440001124820F931F089590E080E00895FC011D
:1014500001900020E9F73197AF01481B590BBC01FF
:101460008DE594E00C949D06FB0101900020E9F7C6
:101470003197AF01461B570B0C94B8091F93CF93BC
:10148000DF93E5E8F1E01281112379F032962181B2
:101490006213F9CFEC016CE50E94A309612FCE0124
:1014A000DF91CF911F910C94A3096111F9CF66E9E7
:1014B00071E0DF91CF911F910C94340A2F923F92EB
:1014C0004F925F926F927F928F929F92AF92BF9254
:1014D000CF92DF92EF92FF920F931F93CF93DF9300
:1014E000CDB7DEB76C970FB6F894DEBF0FBECDBF99
:1014F0008C011B01DC0114968C9114978F77863038
:1015000009F492C268F58230A0F11296ED90FC9039
:101510001397CC901196DC90843008F056C2A70146
:10152000B601C1010E94B809F101828193816C96D4
:101530000FB6F894DEBF0FBECDBFDF91CF911F91E4
:101540000F91FF90EF90DF90CF90BF90AF909F9062
:101550008F907F906F905F904F903F902F90089565
:101560008C3069F160F4883009F459C28A3009F48A
:101570003FC26DE971E0C1010E94340AE5C18032C9
:1015800009F4ECC18034A9F76BE5C1010E94A309FD
:10159000F801008111810115110509F4DAC1B101C9
:1015A000C8010E945E0AC8010E94190A8C01892B99
:1015B00009F4CFC16CE2C1010E94A309ECCFF8018C
:1015C000C080D180E280F380A7019601C701B601F7
:1015D0000E943A258111CDCF20E030E0A901C7015A
:1015E000B6010E943A25882379F0A7019601C70128
:1015F000B6010E94A5269B01AC01C701B6010E945D
:101600003A25882309F4B5CF20E030E0A901C701CD
:10161000B6010E943A2587FF08C06DE2C1010E9411
:10162000A309F7FAF094F7F8F09420E836E948E1D6
:101630005BE4C701B6010E94062887FD81C074E102
:10164000A72EB12C00E210E0188E1F8AF501E65893
:10165000F64F2591359145915491C701B6010E94ED
:10166000062887FD13C0F501E65BF64F25913591FD
:1016700045915491C701B6010E94A0256B017C01E0
:101680002F89388D200F311F388F2F8B1595079597
:1016900034E0A31AB1088CEFA8168FEFB806B1F6A4
:1016A00055245A9420E030E0A901C701B6010E94F8
:1016B000062818160CF04BC02CEA35EC47E257E32D
:1016C000C701B6010E943A2518160CF440C0A52D9A
:1016D000B4E0AB02C0011124B12CA12CFC01EE59E5
:1016E000F64F3F019C012658364F49013FEF5316F4
:1016F00071F1F301EA0DFB1D25913591459154914E
:10170000C701B6010E943A2587FF13C0F401EA0D14
:10171000FB1D2591359145915491C701B6010E9459
:10172000A0256B017C018F89988D801B910B988F70
:101730008F8B159507955A9494E0A91AB108D6CFC6
:1017400000E210E055E0552E188E1F8AABCFC7017E
:10175000B6010E9483274B015C012B013C0106E08E
:1017600080E492E4AFE0B0E0898F9A8FAB8FBC8FBA
:10177000102F01509AE04916510461047104C8F019
:10178000698D7A8D8B8D9C8D2AE030E040E050E0B1
:101790000E941F28298F3A8F4B8F5C8FC301B201A3
:1017A0002AE030E040E050E00E941F2829013A0181
:1017B000DFCFC501B4010E943F259B01AC01C701E9
:1017C000B6010E94A4266B017C01698D7A8D8B8DF8
:1017D0009C8D0E943F259B01AC01C701B6010E9470
:1017E000A0252B013C010E9483276B017C010E94F4
:1017F0003F259B01AC01C301B2010E94A4269B01BD
:10180000AC010E94A5260E948327C60ED71EE81EA3
:10181000F91E898D9A8DAB8DBC8DC816D906EA0646
:10182000FB06D8F09FEF891A990AA90AB90AAF896D
:10183000B88DAB2B39F1BAE08B169104A104B10439
:1018400008F1EF89F88D3196F88FEF8BC12CD12CF0
:101850007601812C912C540183942AE0422E512C44
:10186000612C712CC701B601A30192010E941F28AF
:10187000672B682B692B51F4111644F469017A0126
:101880001150F0CFC12CD12C7601E7CFB501A401C6
:10189000C1010E94CD09112371F14E01F1E18F0EBA
:1018A000911C012F54019AE0492E512C612C712C6E
:1018B000015068F0C701B601A30192010E941F28E0
:1018C000605DD4016E934D0169017A01F1CF812FE2
:1018D00090E0BC0160957095F501E81BF90B31971C
:1018E0008EE2808344275527461B570B6A0D7B1DCC
:1018F000C1010E94B809EF89F88DEF2B29F165E647
:10190000C1010E94A3090F89188D17FF07C06DE25E
:10191000C1010E94A309119501951109FE01779655
:101920009F018AE0E82EF12CC801B7010E940B2824
:10193000805D82938B01672BB9F7A9014E1B5F0B6A
:10194000BF01C1010E94B809D10112968D919C91ED
:10195000EECD6DE5C1010E94A309F6CF6BE7C10191
:101960000E94A309F801008111810115110559F1A7
:10197000D8011696CC9016971796DC9062E2C101BA
:101980000E94A3097601F70161917F01662321F08E
:10199000C1010E943E0AF7CF62E2C1010E94A30981
:1019A0006AE3C1010E94A309B101C8010E945E0A55
:1019B000C8010E94190A8C01892B29F06CE2C1012F
:1019C0000E94A309D2CF6DE7C5CF62E2C1010E9498
:1019D000A3098601E00EF11EE016F10639F0F801C8
:1019E00061918F01C1010E943E0AF6CF62E2B2CF3F
:1019F000CD90DD90ED90FC90B701A601F7FE0BC0F5
:101A00006DE2C1010E94A30944275527BA014C1970
:101A10005D096E097F09C1010E94CD0985CD4D91F7
:101A20005D916D917C91F7CF8C9162EA71E08111AB
:101A300002C067EA71E0C1010E94340A75CDCF92FD
:101A4000DF92EF92FF920F931F93CF93DF93D82FE4
:101A5000C62F0E94F6056B017C018091070381115E
:101A600065C081E080930703809306039FEF909306
:101A70000503109204039C0F909303038093E202EA
:101A80008091E202DD0FD82BD093E2028091E10237
:101A9000813009F07FC01092E1020E94F6056B01CF
:101AA0007C018091E2028093BB00809109039091B8
:101AB0000A03A0910B03B0910C03892B8A2B8B2B6B
:101AC000A1F00E94F6050091090310910A032091EC
:101AD0000B0330910C036C197D098E099F090617C1
:101AE00017072807390708F442C08091BC0083FD1E
:101AF000D8CF85EC8093BC000E94F6056B017C0179
:101B000080910703813009F447C0809104038C174A
:101B100010F4C0910403A3EEB2E0EBEBF2E080E03E
:101B20008C1751F19D9191938F5FFACF80910903AA
:101B300090910A03A0910B03B0910C03892B8A2B7F
:101B40008B2B09F48ACF0E94F605009109031091AE
:101B50000A0320910B0330910C036C197D098E0947
:101B60009F09061717072807390708F076CF8091D5
:101B700008030E941008C0E01092E002C093DF0248
:101B80008C2FDF91CF911F910F91FF90EF90DF90FD
:101B9000CF90089585EEAECF8091090390910A030E
:101BA000A0910B03B0910C03892B8A2B8B2B09F48A
:101BB000A7CF0E94F6050091090310910A03209116
:101BC0000B0330910C036C197D098E099F090617D0
:101BD00017072807390708F093CFC9CFFF920F9353
:101BE0001F93CF93DF93C82F8B0186E70E941C05BC
:101BF0006C2F8EEC93E00E945C090E943108EC2F60
:101C0000E695E77084E0E89FF0011124E151FC4F74
:101C100061817281838194810E941B0686E70E9404
:101C20001C0560E08EEC93E00E945C090E94310884
:101C3000D82F63E086E70E941F0D0E945A05F82EF8
:101C40000E945A05C82F0E945A0530E020E0D1308A
:101C5000C1F0D11119C04C2F50E070E060E0762F38
:101C6000652F542F44276F29482BF8014083518357
:101C700062837383C901DF91CF911F910F91FF9010
:101C8000089521E030E0F6CF22E030E0F3CFFF927C
:101C90000F931F93CF93DF93C82F8B0186E70E948A
:101CA0001C056C2F8EEC93E00E945C090E943108A9
:101CB000EC2FE695E77084E0E89FF0011124EC51E9
:101CC000FC4F64A575A586A597A50E941B0686E70F
:101CD0000E941C0560E08EEC93E00E945C090E946B
:101CE0003108D82F63E086E70E941F0D0E945A0535
:101CF000F82E0E945A05C82F0E945A0530E020E0B5
:101D0000D130C1F0D11119C04C2F50E070E060E02B
:101D1000762F652F542F44276F29482BF8014083D5
:101D2000518362837383C901DF91CF911F910F911A
:101D3000FF90089521E030E0F6CF22E030E0F3CFCD
:101D40000F931F93CF93DF93C82F8B018EE10E94D7
:101D50001C056C2F8EEC93E00E945C090E943108F8
:101D600061E070E080E090E00E941B0663E08EE19D
:101D70000E941F0D0E945A05C82F0E945A05D82F95
:101D80000E945A05C5FD0FC0C2FD10C020E03D2FC6
:101D9000282BF8013183208390E080E0DF91CF9100
:101DA0001F910F91089583E090E0F8CF84E090E0D8
:101DB000F5CF0F931F93CF938C01C62F0E948B09F1
:101DC0006C2F6460C8010E948B096C2F6B7FC80167
:101DD0000E948B0983EC90E00197F1F7CF911F915E
:101DE0000F9108950F931F93CF93DF938C01D62FFC
:101DF000C42F607F642B0E94D90E80E1D89FB00170
:101E000011246C2BC801DF91CF911F910F910C947D
:101E1000D90ECF93DF93CDB7DEB728970FB6F894DE
:101E2000DEBF0FBECDBF98E0E9E0F1E0DE01119624
:101E300001900D929A95E1F790916504981708F436
:101E40008FEF90E0880F991F21E030E02C0F3D1FAD
:101E5000820F931FFC0160816E5F606840E08DE53A
:101E600094E028960FB6F894DEBF0FBECDBFDF9189
:101E7000CF910C94F20E41E00E94F20E81E090E0CE
:101E80000895FC0124813581232B39F421E0FB01E5
:101E90008081882349F020E007C0808191810E94E1
:101EA000AC2B21E0892BB9F7822F08952F923F9216
:101EB0004F925F926F927F928F929F92AF92BF925A
:101EC000CF92DF92EF92FF920F931F93CF93DF9306
:101ED000CDB7DEB7C054D1090FB6F894DEBF0FBE40
:101EE000CDBF9AA789A782E090E00E944E0680E4C9
:101EF0000E941C050E943108811198C386E70E9448
:101F00001C050E943108811191C31092090410929E
:101F1000080480910F04811139C00AE512E080EABB
:101F2000D82E86E70E941C056D2D8EEC93E00E9452
:101F30005C090E943108782E62E086E70E941F0D3E
:101F40000E945A05C82E0E945A057110FFC2FC2C2F
:101F5000E12C4701882AC401D8018D939D938D01FE
:101F6000892B09F4F3C2D394D394BEEADB12D9CF00
:101F700060915B0262956F708AE592E00E946D0548
:101F8000882309F4E3C281E080930F04BE016B5FF4
:101F90007F4F80E50E94470E892B09F0D7C2BE0112
:101FA0006F5F7F4F80E40E94470E892B09F0CEC2FD
:101FB0004D815E816F8178854115510561057105FF
:101FC00009F4C4C289809A80AB80BC808BA69CA691
:101FD000ADA6BEA689288A288B2809F4B7C28091AD
:101FE000640290916502B0E0A0E0BA2FA92F982F6B
:101FF00088274A015B01881A990AAA0ABB0A8D8AB6
:102000009E8AAF8AB88E609166027091670290E0F6
:1020100080E0A50194010E94992807E10E948C2983
:1020200049019A0184010053184F2F4F3F4F0987F0
:102030001A872B873C876D897E898F89988D9B01B4
:10204000AC010E94992889849A84AB84BC8400EDF9
:10205000801607E09006A104B1040CF0ADC2E3E0E5
:10206000AE2EB12CC12CD12CE12CF12C00E010E0D3
:102070000E94412801E20E948C292FA738AB49AB6E
:102080005AAB6BAB7CAB8DAB9EAB89849A84AB8433
:10209000BC84BB0C8808982C5401898A9A8AAB8A24
:1020A000BC8A29853A854B855C856989762F862F80
:1020B000962F205D37404109510961097109810955
:1020C0009109322E432E542E652E762E872E982E71
:1020D000292EADE3AA2EB12C00E00E944128A32CAA
:1020E000B42CC52CD62CE72CF82C092D122D0E94CF
:1020F000412804E00E948C29298F3A8F4B8F5C8FF6
:102100006D8F7E8F8F8F98A3BDE1AB2EB12CC12C2C
:10211000D12CE12CF12C00E010E0232D342D452DA5
:10212000562D672D782D892D922D0E944128A32CA4
:10213000B42CC52CD62CE72CF82C092D122D0E947E
:10214000412804E00E948C2929A33AA34BA35CA355
:102150006DA37EA38FA398A789849A84AB84BC8443
:1021600004E280160AEF90060FEFA006B0060CF00E
:102170006EC029853A854B855C856989762F862FC7
:10218000962F24523A4F4F4F5F4F6F4F7F4F8F4FD5
:102190009F4F322E432E542E652E762E872E982E4C
:1021A000292E01E1A02EB12CC12CD12CE12CF12C37
:1021B00000E010E00E944128A32CB42CC52CD62CA2
:1021C000E72CF82C092D122D0E944128A98CBA8CDD
:1021D000CB8CDC8CED8CFE8C0F8D18A10E94A92974
:1021E000298F3A8F4B8F5C8F6D8F7E8F8F8F98A347
:1021F00089E0A82EB12CC12CD12CE12CF12C00E0CF
:1022000010E0232D342D452D562D672D782D892D49
:10221000922D0E944128A32CB42CC52CD62CE72C3F
:10222000F82C092D122D0E944128A9A0BAA0CBA0FC
:10223000DCA0EDA0FEA00FA118A50E94A92929A34A
:102240003AA34BA35CA36DA37EA38FA398A7609131
:1022500062027091630290E080E02D893E894F898F
:10226000588D0E94992806E00E948C2939014A0164
:10227000B62FA72FF82FE92FA0905E02B0905F0233
:10228000950140E050E060E070E080E090E001E126
:102290000E94732959016A017B018C019301A401F9
:1022A0006B2F7A2F8F2F9E2F0E94A929522E432EFB
:1022B0004FAB58AF69AF7AAF8BAF9CAF6091600204
:1022C0007091610290E080E02D893E894F89588DA0
:1022D0000E94992807E00E948C2939014A01B62FF3
:1022E000A72FF82FE92FA0905C02B0905D02950116
:1022F00040E050E060E070E080E090E000E10E94AB
:10230000732959016A017B018C019301A4016B2F90
:102310007A2F8F2F9E2F0E94A92959016A017B01D4
:102320008C0169857A858B859C850E9441253B01BE
:102330004C012FA538A949A95AA96BA97CA98DA937
:102340009EA90E94B2279B01AC01C401B3010E9467
:10235000A42620E030E048EC52E40E941127698B6B
:102360007D8B382E292E9501A601B701C801A9A0A1
:10237000BAA0CBA0DCA0EDA0FEA00FA118A50E94E2
:10238000B229ABA4BCA4CDA4DEA445015601C12C46
:10239000D12C760189869A86AB86BC86CD86DE8670
:1023A000EF86F88A5401CB84DC84E12CF12C00E028
:1023B00010E00E94412805E10E948C2939014A0160
:1023C000B62FA72FF82FE92F252D342D4FA958AD63
:1023D00069AD7AAD8BAD9CADA98CBA8CCB8CDC8C05
:1023E000ED8CFE8C0F8D18A10E94B22959016A0153
:1023F0007B018C019301A4016B2F7A2F8F2F9E2FCD
:102400000E94B2290FE00E948C290E94B22720E08E
:1024100030E048EC52E40E941127698F7A8F8B8F4D
:102420009C8F80E40E941C0580910804909109040F
:10243000892B09F0E8C065EE8EEC93E00E945C0900
:102440000E943108F82E63E080E40E941F0D0E9474
:102450005A05082F0E945A05182F0E945A05482F26
:10246000BB24B394FB1409F471C0F1106FC060E099
:10247000702F612B90E080E00027162F272F382F38
:10248000E0E1F0E0C12C50E8D52EEE24EA94F12CE6
:10249000CBA6DCA6EDA6FEA6C12CA0E8DA2EA8E904
:1024A000EA2EF12C412C512CB0E86B2E712C5301EB
:1024B000420180229122A222B32289288A288B28D5
:1024C00061F08BA49CA4ADA4BEA48C209D20AE2062
:1024D000BF20082519252A253B2576946794579413
:1024E00047948BA49CA4ADA4BEA4B694A79497943F
:1024F00087948BA69CA6ADA6BEA6F694E794D79427
:10250000C7943197A1F6C42ED12CF12CE12CC01622
:10251000D106E206F306D1F40E943F2520E030E028
:102520004AEF52E40E94A02520E030E040E857E363
:102530000E94A02520E030E040EC50E40E94A42658
:102540006DAF7EAF8FAF21969FAF219767E072E0AE
:1025500089A59AA50E94410F811110C06DEA71E012
:1025600089A59AA50E94410F811168C062EB71E0B4
:1025700089A59AA50E94410F811169C069897D8949
:10258000832D922DC05CDF4F0FB6F894DEBF0FBED7
:10259000CDBFDF91CF911F910F91FF90EF90DF9012
:1025A000CF90BF90AF909F908F907F906F905F90F3
:1025B0004F903F902F90089515E0A12EB12CC12C83
:1025C000D12CE12CF12C00E010E00E94412806E221
:1025D0000E948C292FA738AB49AB5AAB6BAB7CABB5
:1025E0008DAB9EAB19A21AA21BA21CA21DA21EA2F9
:1025F0001FA218A6198E1A8E1B8E1C8E1D8E1E8E63
:102600001F8E18A224CE65EF8EEC93E00E945C0929
:102610000E943108F82E60910A0470910B04809199
:102620000C0490910D040E941B060DCF80E00E94C7
:10263000090F87EB91E00E94270AA0CF9DAC998AF1
:102640008EAC8D8A3FAC21962FAC219797CF998C79
:10265000998AAA8CAD8A3B8C2C8C90CF2F923F927A
:102660004F925F926F927F928F929F92AF92BF92A2
:10267000CF92DF92EF92FF920F931F93CF93DF934E
:10268000CDB7DEB7ED970FB6F894DEBF0FBECDBF66
:102690009EA78DA781E090E00E944E0686E70E94EB
:1026A0001C050E9431088111DEC28091ED03811169
:1026B00038C00DED13E030EA532E86E70E941C056A
:1026C000652D8EEC93E00E945C090E943108382E43
:1026D00062E086E70E941F0D0E945A05482E0E9464
:1026E0005A0521E0321609F46CC2F42CE12CD70112
:1026F000A82BCD01F801819391938F0153945394AA
:10270000FEEA5F12DACF6091DE0362956F708DEDA5
:1027100093E00E946D05882309F453C281E0809301
:10272000ED038091EE03880FBE016B5F7F4F8065E4
:102730000E94EE0D892B09F044C28091EE03880FB0
:10274000BE016F5F7F4F80640E94EE0D892B09F000
:1027500038C24D815E816F817885411551056105D3
:10276000710509F42EC2E980FA800B811C81E9A66B
:10277000FAA60BA71CA7EF28E02AE12A09F421C238
:102780008091E7039091E803B0E0A0E0BA2FA92F71
:10279000982F88278A019B01081B190B2A0B3B0BDA
:1027A0000D8B1E8B2F8B388F6091E9037091EA039C
:1027B00090E080E0A90198010E94992807E10E9419
:1027C0008C29DA01C9018053984FAF4FBF4F8987D9
:1027D0009A87AB87BC876D897E898F89988D9B018D
:1027E000AC010E949928A984BA84CB84DC8400EDD2
:1027F000A01607E0B006C104D1040CF00DC2B3E08E
:10280000AB2EB12CC12CD12CE12CF12C00E010E02E
:102810000E94412801E20E948C292FA738AB49ABC6
:102820005AAB6BAB7CAB8DAB9EAB89859A85AB8588
:10283000BC85BB0F880B982FDC01898B9A8BAB8BE7
:10284000BC8B29853A854B855C856989762F862FD7
:10285000962F205D374041095109610971098109AD
:102860009109322E432E542E652E762E872E982EC9
:10287000292E8DE3A82E00E0232D342D452D562D35
:10288000672D782D892D922D0E944128A32CB42CE0
:10289000C52CD62CE72CF82C092D122D0E9441288E
:1028A00004E00E948C29298F3A8F4B8F5C8F6D8FAB
:1028B0007E8F8F8F98A39DE1A92EB12CC12CD12C96
:1028C000E12CF12C00E010E0232D342D452D562D68
:1028D000672D782D892D922D0E944128A32CB42C90
:1028E000C52CD62CE72CF82C092D122D0E9441283E
:1028F00004E00E948C2929A33AA34BA35CA36DA3F7
:102900007EA38FA398A7A984BA84CB84DC8404E235
:10291000A0160AEFB0060FEFC006D0060CF06EC08E
:1029200029853A854B855C856989762F862F962F78
:1029300024523A4F4F4F5F4F6F4F7F4F8F4F9F4FF4
:10294000322E432E542E652E762E872E982E292E2B
:10295000F1E1AF2EB12CC12CD12CE12CF12C00E0F7
:1029600010E00E944128A32CB42CC52CD62CE72CB7
:10297000F82C092D122D0E944128A98CBA8CCB8CE1
:10298000DC8CED8CFE8C0F8D18A10E94A929298F5B
:102990003A8F4B8F5C8F6D8F7E8F8F8F98A3A9E0BE
:1029A000AA2EB12CC12CD12CE12CF12C00E010E08E
:1029B000232D342D452D562D672D782D892D922DC3
:1029C0000E944128A32CB42CC52CD62CE72CF82C23
:1029D000092D122D0E944128A9A0BAA0CBA0DCA0ED
:1029E000EDA0FEA00FA118A50E94A92929A33AA332
:1029F0004BA35CA36DA37EA38FA398A76091E5036F
:102A00007091E60390E080E02D893E894F89588DD2
:102A10000E94992806E00E948C2939014A01B62FAC
:102A2000A72FF82FE92FA090E103B090E2039501C2
:102A300040E050E060E070E080E090E001E10E9462
:102A4000732959016A017B018C019301A4016B2F49
:102A50007A2F8F2F9E2F0E94A929298B3FAB48AF39
:102A600059AF6AAF7BAF8CAF9DAF6091E3037091BC
:102A7000E40390E080E02D893E894F89588D0E94C3
:102A8000992807E00E948C2939014A01B62FA72F07
:102A9000F82FE92FA090DF03B090E003950140E00C
:102AA00050E060E070E080E090E000E10E94732977
:102AB00059016A017B018C019301A4016B2F7A2FCC
:102AC0008F2F9E2F0E94A92979018A011B012C01B9
:102AD00069857A858B859C850E9441254B015C0127
:102AE0002FA538A949A95AA96BA97CA98DA99EA986
:102AF0000E94B2279B01AC01C501B4010E94A4262B
:102B000020E030E048EC52E40E9411273B014C01E8
:102B10009701A801B101C201A9A0BAA0CBA0DCA075
:102B2000EDA0FEA00FA118A50E94B229C9A4DAA4A5
:102B3000EBA4FCA456016701E12CF12C8701A986C6
:102B4000BA86CB86DC86ED86FE860F87188BE12C55
:102B5000F12C00E010E00E94412805E10E948C2940
:102B600019012A01B62FA72FF82FE92F29893FA98C
:102B700048AD59AD6AAD7BAD8CAD9DADA98CBA8C1D
:102B8000CB8CDC8CED8CFE8C0F8D18A10E94B229B1
:102B900059016A017B018C019101A2016B2F7A2FEF
:102BA0008F2F9E2F0E94B2290FE00E948C290E9435
:102BB000B22720E030E048EC52E40E9411275B018C
:102BC0006C0167E072E08DA59EA50E94410F811106
:102BD00008C062EB71E08DA59EA50E94410F811196
:102BE0004AC0B301C401ED960FB6F894DEBF0FBE24
:102BF000CDBFDF91CF911F910F91FF90EF90DF90AC
:102C0000CF90BF90AF909F908F907F906F905F908C
:102C10004F903F902F900895E5E0AE2EB12CC12C3F
:102C2000D12CE12CF12C00E010E00E94412806E2BA
:102C30000E948C292FA738AB49AB5AAB6BAB7CAB4E
:102C40008DAB9EAB19A21AA21BA21CA21DA21EA292
:102C50001FA218A6198E1A8E1B8E1C8E1D8E1E8EFC
:102C60001F8E18A2CBCE80E00E94090F8AEC91E063
:102C70000E94270AB6CF35014601B3CF2F923F926B
:102C80004F925F926F927F928F929F92AF92BF927C
:102C9000CF92DF92EF92FF920F931F93CF93DF9328
:102CA000CDB7DEB760970FB6F894DEBF0FBECDBFCD
:102CB00098878F8390E080E00E944E0680E40E9417
:102CC0001C050E9431088111F7C01092DB0310929D
:102CD000DA0380E40E941C0563EF8EEC93E00E940F
:102CE0005C090E94310862E370E080E090E00E949D
:102CF0001B0663E080E40E941F0D0E945A05082F06
:102D00000E945A05182F0E945A05482F60E0702F24
:102D1000612B90E080E00027162F272F382FE0E16D
:102D2000F0E0812C50E8952EAA24AA94B12CC12C55
:102D3000A0E8DA2EA8E9EA2EF12CCD86DE86EF8611
:102D4000F88A412C512CB0E86B2E712C7301620172
:102D5000C022D122E222F322CD28CE28CF2861F052
:102D6000CD84DE84EF84F888C820D920EA20FB20B7
:102D70000C251D252E253F2576946794579447945E
:102D8000B694A79497948794CD84DE84EF84F888D2
:102D9000F694E794D794C794CD86DE86EF86F88ABA
:102DA0003197A1F6842E912CB12CA12C801691067E
:102DB000A206B30609F053C00E943F2522E538EB76
:102DC0004FE253E40E94A02520E030E040E857E3C2
:102DD0000E94A02526E636E64BE352E40E94A42694
:102DE00069837A838C879B8780E40E941C0565EF4A
:102DF0008EEC93E00E945C090E94310862E370E06F
:102E000080E090E00E941B0663E080E40E941F0DBA
:102E10000E945A05082F0E945A05182F0E945A0531
:102E20000E94310860E0702F612B90E080E00E94EA
:102E30003F2520E030E04AEF52E40E94A02520E048
:102E400030E040E857E30E94A02520E030E040EC6D
:102E500050E40E94A42669877A87382E292E67E0DD
:102E600072E08F8198850E94410F811108C06DEA40
:102E700071E08F8198850E94410F811125C0698181
:102E80007A818C859B8560960FB6F894DEBF0FBE65
:102E9000CDBFDF91CF911F910F91FF90EF90DF9009
:102EA000CF90BF90AF909F908F907F906F905F90EA
:102EB0004F903F902F90089580E00E94090F8DED74
:102EC00091E00E94270ADBCFD984D982EA84EA8282
:102ED0003C862B86D4CFCF92DF92EF92FF920F9356
:102EE0001F93CF93DF93FC018481982F9F7739F450
:102EF000807880628483118210821382128284819E
:102F000085FD0BC080E090E0DF91CF911F910F9184
:102F1000FF90EF90DF90CF9008956115710591F3C8
:102F2000EA017B016F01008111810115110589F111
:102F3000D80116966D917C91C7010E94AC2B892B0C
:102F400031F1C8010E94190A8C01EFCF3897FD8337
:102F5000EC833097B9F2E601AA81BB81109791F01A
:102F6000CF018A1B9B0B23E0959587952A95E1F766
:102F700015968C93FB83EA8315821482F782E6828E
:102F8000CF01C2CFF983E883FB83EA83F5CFC80181
:102F9000BBCFEC81FD818A819B810896E817F907F8
:102FA000A8F681E08887AECF0F931F93CF93DF936E
:102FB000EC0188819981009759F02A813B8126177D
:102FC000370730F081E0DF91CF911F910F91089585
:102FD0008B016F5F7F4F0E94E62A009759F099831B
:102FE00088831B830A832C813D81232B59F7FC01A5
:102FF0001082E8CF80E0E7CFEF92FF920F931F930C
:10300000CF93DF936115710541F480E0DF91CF919B
:103010001F910F91FF90EF90089541155105B1F068
:103020007B01EC010C811D81040F151FB8010E946A
:10303000D417882351F3288139818C819D81B70170
:10304000820F931F0E94B52B1D830C8381E0DECF7E
:10305000CF93DF93EC0188819981009711F00E9452
:103060005D2A198218821D821C821B821A82DF91BE
:10307000CF910895CF93DF93EC01FB0101900020E5
:10308000E9F73197AF01461B570B0E94FC178111DE
:1030900003C0CE010E942818CE01DF91CF91089580
:1030A000CF93DF93EC01FB014481558160817181F5
:1030B0000E94FC17811103C0CE010E942818CE0186
:1030C000DF91CF910895EF92FF920F931F93CF93CB
:1030D000DF93EC017B018A01BA010E94D4178111B0
:1030E0000BC0CE010E942818CE01DF91CF911F9115
:1030F0000F91FF90EF9008951D830C83B701888195
:1031000099810E94B52BF0CFEF92FF920F931F93FE
:10311000CF93DF93CDB7DEB7A1970FB6F894DEBF9C
:103120000FBECDBF7C01CB01BA01F7011182108225
:1031300013821282158214828E010F5F1F4F22E0CC
:1031400044E00E94E5220097C9F0FC0101900020B4
:10315000E9F73197AF01481B590BBC01C7010E9429
:103160006318A1960FB6F894DEBF0FBECDBFDF91F6
:10317000CF911F910F91FF90EF900895C7010E948A
:103180002818EFCFFB01DC0111961C921E921396BA
:103190001C921E92129715961C921E9214978617D7
:1031A000970749F0608171816115710521F04481B3
:1031B00055810C9463180895FC01118210821382CA
:1031C000128215821482FB0101900020E9F73197E9
:1031D000AF01461B570B0C946318FC018081918151
:1031E000009711F00C945D2A08952F923F924F9210
:1031F0005F926F927F928F929F92AF92BF92CF9287
:10320000DF92EF92FF920F931F93CF93DF93CDB78F
:10321000DEB7CF54D1090FB6F894DEBF0FBECDBFD5
:103220008C0167E072E00E94410F882309F463C4B7
:1032300067E072E0CE0180960E94DC18CE01809695
:103240000E943E162B013C0167E072E0CE014A96D7
:103250000E94DC18CE014A960E942E139B01AC01FD
:10326000C301B2010E94A5262B013C0167E072E078
:10327000CE0144960E94DC18CE0144960E94560F5F
:103280009B01AC01C301B2010E94A5262B013C01A8
:1032900067E072E0CE010E960E94DC1883E090E0B9
:1032A0000E944E06809128040E941C050E9431084D
:1032B00081110FC480914D0481112CC05DE3A52EB6
:1032C00054E0B52E10EA809128040E941C05612F5D
:1032D0008EEC93E00E945C090E943108E82E62E0C7
:1032E000809128040E941F0D0E945A05082F0E94F9
:1032F0005A05E110A1C0902E812C9401282BC90100
:10330000D5018D939D935D011E5F103BE1F681E039
:1033100080934D04809128040E941C0568E48EEC83
:1033200093E00E945C090E9431086AE070E080E04E
:1033300090E00E941B06809128040E941C0560E01A
:103340008EEC93E00E945C090E94310863E080915A
:1033500028040E941F0D0E945A05082F0E945A053A
:10336000182F0E945A05612F70E090E080E0982F9E
:10337000872F762F6627802B672F782F892F992705
:103380000E943F2520E030E543EC57E40E941127DE
:103390006B017C010DE314E01FA30EA30FE314E007
:1033A000812C912C5401D8016D917D918D0190E07B
:1033B00080E00E943F25EEA1FFA1529142913291FF
:1033C0002291FFA3EEA30E94A025A50194010E94D3
:1033D000A526A70196010E94A0254B015C0127E4C8
:1033E00034E020173107F9F620E030E040E251E404
:1033F0000E94A0254B015C01609147047091480434
:1034000090E080E00E943F252091290430912A0419
:1034100040912B0450912C040E94A025A5019401F9
:103420000E94A52620E030E048EC52E40E941127DB
:103430006EA3C72ED82EF92E67E072E0CE010E964D
:103440000E94410F882329F0AEA0ACA6C8AADCAA2E
:10345000F8AE2CA538A94CA958ADC301B2010E9401
:10346000A52668AF79AF8AAF9BAF6E0108E0C00EAA
:10347000D11C67E072E0C6010E94DC1884E090E095
:103480000E944E068EE10E941C050E9431088111A7
:103490002AC380914E0481113AC06FE474E00E9407
:1034A000A00E892B09F0B8C261E574E081E00E94AA
:1034B000A00E892B09F0B0C263E574E08AE10E9496
:1034C000A00E892B09F0A8C265E574E08BE10E948B
:1034D000A00E892B09F0A0C267E574E08CE10E9480
:1034E000A00E892B09F098C269E574E08DE10E9475
:1034F000A00E892B09F090C26BE574E08CE20E946B
:10350000A00E892B09F088C281E080934E048EE1E1
:103510000E941C056FEA8EEC93E00E945C090E94F9
:103520003108F82E64E670E080E090E00E941B060F
:1035300067E08EE10E941F0D8E010F5F1F4F0E94FA
:103540005A05D8018D938D01CA16DB06C1F7F1101B
:1035500063C28981847209F05FC2AA80AEA21B8116
:103560000C818D818E80912CB12CA12CBA2CA92C90
:10357000982C8824A82A8F81882A609153047091FE
:103580005404072E000C880B990B0E9441252B0137
:103590003C016091550470915604072E000C880B75
:1035A000990B0E944125A30192010E94A4266B0160
:1035B0007C01C501B4010E94412520E030E040E8D3
:1035C00053E30E94A0259B01AC01C701B6010E94F4
:1035D000A025A30192010E94A5266AA77BA71C0132
:1035E0002AEB822E21E0922EF4016591759185914E
:1035F00094910E9441259B01AC016AA57BA5C10164
:103600000E94062818160CF007C2E2EFF8E0659158
:103610007591859194910E9441259B01AC016AA509
:103620007BA5C1010E943A2518160CF4F5C1662449
:103630006394712C562CF401659175918591949148
:103640000E9441259B01AC016AA57BA5C1010E9496
:103650000628181684F4C401885A9F4F2FEF621A67
:10366000720A39E16316710409F03BC2A8E16A2EBF
:10367000712CB8E15B2E612F70E090E080E0982F14
:10368000872F762F6627AEA08A29602B8058910954
:1036900020915B0430915C04032E000C440B550B0D
:1036A0000E949928E8EEAE2EF3E0BF2EC12CD12C5B
:1036B000E12CF12C00E010E00E94D5282EA33FA3BE
:1036C00048A759A75A9406E1509E7001112441E081
:1036D00050E0442ED701A40FB51FAA0FBB1FAA0F9D
:1036E000BB1FAE59BE4FFD016591759185919491B7
:1036F000AEA0BFA0C8A4D9A46A157B058C059D0502
:103700004CF44F5F5F4F4831510519F747E150E0E6
:1037100087E1482E86E1869DB001879D700D1124BA
:1037200081E090E08CAB3B01680E791E660C771C43
:10373000660C771C83010E591E4F3801F801A590C5
:10374000B590C590D4900EA11FA128A539A5A016AB
:10375000B106C206D30644F401968831910511F7EB
:1037600087E190E017E11CAB28E5529EF00111249F
:10377000EE59FE4FA590B590C590D490ACA6BDA6CD
:10378000CEA6DFA6F401A590B590C590D490ACAEBE
:10379000BDAECEAEDFAE0FEF040D10E0F801EE0DC2
:1037A000FF1DEE0FFF1FEE0FFF1FEE59FE4FC590DE
:1037B000D590E590F490C8AAD9AAEAAAFBAAFD017F
:1037C000A590B590C590D4902496ACAEBDAECEAECB
:1037D000DFAE24972CA9215030E0F901E60FF71F46
:1037E000EE0FFF1FEE0FFF1FEE59FE4FC590D59055
:1037F000E590F490CCAADDAAEEAAFFAAF301A59069
:10380000B590C590D4902896ACAEBDAECEAEDFAE2E
:103810002897F801EE0FFF1FEE0FFF1FEE59FE4F26
:10382000C590D590E590F490FA01EE0FFF1FEE0FD2
:10383000FF1FEE59FE4F45915591659174912C965D
:103840004CAF5DAF6EAF7FAF2C97F901EE0FFF1F4E
:10385000EE0FFF1FEE59FE4F85909590A590B49006
:10386000FC01EE0FFF1FEE0FFF1FEE59FE4F65919B
:1038700075918591949160966CAF7DAF8EAF9FAF3F
:1038800060976EA17FA188A599A508A919A92AA961
:103890003BA9601B710B820B930B0E9441252B01EE
:1038A0003C0124966CAD7DAD8EAD9FAD249728A9CB
:1038B00039A94AA95BA9621B730B840B950B0E9463
:1038C00041259B01AC01C301B2010E9411272B01CC
:1038D0003C012C966CAD7DAD8EAD9FAD2C976C19D7
:1038E0007D098E099F090E9441259B01AC01C301FE
:1038F000B2010E94A0252B013C01C701B6010E9424
:1039000041259B01AC01C301B2010E94A5266B01B8
:103910007C016EA17FA188A599A50CA91DA92EA93E
:103920003FA9601B710B820B930B0E9441252B0159
:103930003C0128966CAD7DAD8EAD9FAD28972CA92E
:103940003DA94EA95FA9621B730B840B950B0E94C6
:1039500041259B01AC01C301B2010E9411272B013B
:103960003C0160966CAD7DAD8EAD9FAD60976819E2
:1039700079098A099B090E9441259B01AC01C30179
:10398000B2010E94A0252B013C01C501B4010E9497
:1039900041259B01AC01C301B2010E94A526A701EC
:1039A00096010E94A4264B015C016CA57DA58EA505
:1039B0009FA50E9441259B01AC016AA57BA5C10181
:1039C0000E94A4262B013C016CAD7DAD8EAD9FAD58
:1039D0000CA51DA52EA53FA5601B710B820B930B9B
:1039E0000E9441259B01AC01C301B2010E94112735
:1039F0009B01AC01C501B4010E94A025A70196015D
:103A00000E94A5266CAF21967FAF219725968FAF98
:103A1000259729969FAF299767E072E0CE01089617
:103A20000E94410F811114C063E072E0CE0108963C
:103A30000E94410F882361F01CAD1AA72196AFACFC
:103A40002197ABA625962FAC259729963FAC2997B1
:103A50002AA53BA5A10168AD79AD8AAD9BAD0E94B9
:103A6000A52620E030E040EA50E40E9411276B01D7
:103A70007C01CE0108960E94ED18CE010E960E94A0
:103A8000ED18CE0144960E94ED18CE014A960E9490
:103A9000ED18CE0180960E94ED18C701B601C15BFA
:103AA000DF4F0FB6F894DEBF0FBECDBFDF91CF91D1
:103AB0001F910F91FF90EF90DF90CF90BF90AF904C
:103AC0009F908F907F906F905F904F903F902F903E
:103AD000089580E00E94090F80EF91E00E94270A7C
:103AE000B8CC4C01A7CD80E00E94090F8CE092E099
:103AF0000E94270AADCF6DEA71E0C8010E94410F14
:103B0000882359F16DEA71E0CE0108960E94DC1815
:103B1000CE0108960E943E166B017C016DEA71E0B1
:103B2000CE0101960E94DC18CE0101960E94560F2C
:103B30009B01AC01C701B6010E94A52620E030E040
:103B400040E05FE30E94A0256B017C01CE0101965D
:103B50000E94ED18CE0108969ECF62EB71E0C8017D
:103B60000E94410F882309F498CF62EB71E0CE01E7
:103B700008960E94DC18CE0108960E94560F6B0131
:103B80007C0162EB71E0CE0101960E94DC18CE014F
:103B900001960E942E13CCCF85ED8093BC008091BE
:103BA000090390910A03A0910B03B0910C030796AF
:103BB000A11DB11D23E0B695A795979587952A95E8
:103BC000D1F72091BC0024FD03C010920703089593
:103BD0004091090350910A0360910B0370910C030B
:103BE000452B462B472B69F30097A105B10541F002
:103BF0002AE22A95F1F700C00197A109B109E1CFA6
:103C0000809108030C9410081F920F920FB60F9228
:103C100011242F933F938F939F93AF93BF938091E2
:103C2000B3029091B402A091B502B091B602309166
:103C3000B20223E0230F2D3758F50196A11DB11DC7
:103C40002093B2028093B3029093B402A093B50282
:103C5000B093B6028091B7029091B802A091B902D8
:103C6000B091BA020196A11DB11D8093B702909345
:103C7000B802A093B902B093BA02BF91AF919F91DD
:103C80008F913F912F910F900FBE0F901F9018951D
:103C900026E8230F0296A11DB11DD2CF1F920F92CD
:103CA0000FB60F9211242F933F934F935F936F930F
:103CB0007F938F939F93AF93BF93EF93FF9381E392
:103CC00093E00E942407FF91EF91BF91AF919F91E4
:103CD0008F917F916F915F914F913F912F910F90B5
:103CE0000FBE0F901F9018951F920F920FB60F9254
:103CF00011242F938F939F93EF93FF93E0914103B0
:103D0000F09142038081E0914703F091480382FDE6
:103D10001BC0908180914A038F5F8F7320914B036A
:103D2000821741F0E0914A03F0E0EF5CFC4F958F81
:103D300080934A03FF91EF919F918F912F910F9064
:103D40000FBE0F901F9018958081F4CF1F920F9295
:103D50000FB60F9211242F933F934F935F936F935E
:103D60007F938F939F93AF93BF93EF93FF93809134
:103D7000B900887F803609F44AC0F0F5883209F42A
:103D8000A7C018F5803109F49BC0B8F4882309F462
:103D9000F9C0883009F494C0FF91EF91BF91AF91C1
:103DA0009F918F917F916F915F914F913F912F9153
:103DB0000F900FBE0F901F901895883109F488C09E
:103DC000803251F78093050314C0803409F49DC0FC
:103DD00040F48033B9F38833F9F68093050385EC1A
:103DE000B0C0803509F485C0883509F496C08834A0
:103DF00099F60E94CC1DD0CF883909F48CC038F5D3
:103E0000883729F050F4883611F0803729F683E09E
:103E1000809307031092AD0257C0883809F47BC025
:103E2000803919F0803809F0B7CF8091AD02803227
:103E300008F071C0E091AD0281E08E0F8093AD0279
:103E40008091BB00F0E0E357FD4F80833DC0803B95
:103E500039F0E0F4803A09F479C0883A09F09CCF4F
:103E600084E08093070310928C0210928B02E09101
:103E7000DD02F091DE02099580918B0281110FC065
:103E800081E080938B0210926B0209C0803C09F4A0
:103E9000A6CF883C09F4A3CF883B09F07DCFE09101
:103EA0008C0281E08E0F80938C02F0E0E559FD4F8B
:103EB00080818093BB0090918C0280918B0229C0FD
:103EC0008091E2028093BB0085EC8093BC0064CFBC
:103ED0009091040380910303981758F5E09104032F
:103EE00081E08E0F80930403F0E0ED51FD4F80815F
:103EF000E9CFE091040381E08E0F80930403809169
:103F0000BB00F0E0ED51FD4F808390910403809160
:103F100003039817C8F285E8D8CFE091040381E045
:103F20008E0F809304038091BB00F0E0ED51FD4FB4
:103F300080838091060381115CCF81E08093E10250
:103F400084EA8093BC001092070326CF85EC80930F
:103F5000BC00109207038091AD02803230F4E091F2
:103F6000AD02F0E0E357FD4F10826091AD0270E0CA
:103F7000E091DB02F091DC028DE892E0099510926D
:103F8000AD020ACF1092050334CFCF93DF93E1E364
:103F9000F3E01382128288EE93E0A0E0B0E0848325
:103FA0009583A683B78329E531E03183208325EC0F
:103FB00030E03587248724EC30E03787268720ECF3
:103FC00030E0318B208B21EC30E0338B228B22ECE4
:103FD00030E0358B248B26EC30E0378B268B118E2E
:103FE000128E138E148EEEECF3E013821282848311
:103FF0009583A683B7838BE691E091838083EDE57B
:10400000F4E0138212828DE791E09183808387E24E
:10401000848380E1818782E0828713861092DB03AC
:104020001092DA03CCEDD3E0198A88E1E1E1F1E006
:10403000A0EFB3E001900D928A95E1F788E1E9E203
:10404000F1E0A0E1B4E001900D928A95E1F780EAF9
:1040500090E0A0E0B0E08EA79FA7A8ABB9AB81E04D
:1040600090E09DA78CA71AAA1BAA87E78093280433
:1040700084E1E1E4F1E0A9E2B4E001900D928A95D7
:10408000E1F710924D0410924E04DF91CF91089504
:10409000CF93DF93CDB7DEB7CA58D1090FB6F894E6
:1040A000DEBF0FBECDBF789484B5826084BD84B579
:1040B000816084BD85B5826085BD85B5816085BD23
:1040C00080916E00816080936E00109281008091DB
:1040D0008100826080938100809181008160809363
:1040E0008100809180008160809380008091B10088
:1040F00084608093B1008091B00081608093B000B3
:1041000080917A00846080937A0080917A00826046
:1041100080937A0080917A00816080937A00809108
:104120007A00806880937A001092C100E091410388
:10413000F091420382E08083E0913D03F0913E03E1
:104140001082E0913F03F09140038FEC8083109246
:104150004903E0914503F091460386E08083E091B6
:104160004303F0914403808180618083E0914303A5
:10417000F0914403808188608083E0914303F09153
:104180004403808180688083E0914303F09144037D
:1041900080818F7D808385E090E00E944E060E94A2
:1041A000F9070E94F9070E94F9070E94F9070E9487
:1041B000F9070E94F9071092620480916704823027
:1041C00018F098E0909362048093650462E370E0D5
:1041D00080E090E00E941B06609168048DE594E009
:1041E0000E948B0968EE73E080E090E00E941B065D
:1041F00060E38DE594E00E94D90E0BE416E4C8015B
:104200000197F1F760E38DE594E00E94D90EC801B3
:104210000197F1F760E38DE594E00E94D90E83E504
:1042200092E00197F1F760E28DE594E00E94D90EEB
:1042300060916204606240E08DE594E00E94F20EBD
:1042400084E08093630440E06CE08DE594E00E949C
:10425000F20E40E061E08DE594E00E94F20E0BE387
:104260001FE1C8010197F1F782E08093640440E008
:1042700066E08DE594E00E94F20E40E062E08DE59C
:1042800094E00E94F20EC8010197F1F788E0809354
:10429000680460E08DE594E00E948B091E012FE028
:1042A000220E311C8E010D581F4F2FB7F8948091AC
:1042B000B3029091B402A091B502B091B6022FBFA3
:1042C0004091AE025091AF026091B0027091B10284
:1042D0006C017D01C41AD50AE60AF70AB701A601E6
:1042E000403157426105710508F404C18093AE0264
:1042F0009093AF02A093B002B093B1023A822982A8
:104300003C822B821E830D8318870F8319861E869D
:1043100067E072E0C8010E94DC18C8010E94F5182D
:104320002B013C01C8010E94ED1862EB71E0C8014D
:104330000E94DC18C8010E94F5186B017C01C801BD
:104340000E94ED186DEA71E0C8010E94DC18C801F6
:104350000E94F5184B015C01C8010E94ED18809184
:10436000010190910201019709F073C040E061E002
:104370008DE594E00E94F20E8BE39FE10197F1F747
:10438000B301A201C8010E9484186FE172E0CE015E
:1043900087589F4F0E94DC18B801CE0187589F4F65
:1043A0000E94501863E272E00E943A18BC01CE01EC
:1043B0008B579F4F0E94C218CE0187589F4F0E9473
:1043C000ED18C8010E94ED1880E00E94090FCE018F
:1043D0008B579F4F0E94CA0680910001882309F4E1
:1043E000B8C0B501A401C8010E94841866E272E059
:1043F000CE0187589F4F0E94DC18B801CE01875824
:104400009F4F0E9450186AE272E00E943A18BC0165
:10441000CE0181589F4F0E94C218CE0187589F4FEE
:104420000E94ED18C8010E94ED1881E00E94090F5A
:10443000CE0181589F4F0E94CA0610920001CE0102
:1044400081589F4F0E94ED18CE018B579F4F0E94BD
:10445000ED18AE014F5F5F4F68E372E0CE010A9640
:104460000E946B17FC01892B41F0948190789C602D
:1044700094834082518262827382AE014F5F5F4FAC
:1044800064E472E0CE010A960E946B17FC01892B4E
:1044900041F0948190789C60948380829182A28282
:1044A000B382AE014F5F5F4F6DE472E0CE010A96BA
:1044B0000E946B17FC01892B41F0948190789C60DD
:1044C0009483C082D182E282F38221E3C22E23E070
:1044D000D22EF801D182C08213821282B801CE019D
:1044E0000A960E945E0A42E050E066E572E0C6016C
:1044F0000E949D0681E393E00E94930781E393E08D
:104500000E94E20684359105B9F4809101019091F1
:104510000201892B09F04DC088E0D82ED0926804A2
:1045200060E08DE594E00E948B09EE24E394F12C89
:10453000F0920201E092010180E090E0892B09F401
:10454000B4CE0E941007882309F4AFCE0E94000069
:10455000ACCEB701A601C8010E9484186FE272E0D8
:10456000CE0187589F4F0E94DC18B801CE018758B2
:104570009F4F0E94501863E372E00E943A18BC01FA
:10458000CE0181589F4F0E94C218CE0187589F4F7D
:104590000E94ED18C8010E94ED1881E00E94090FE9
:1045A000CE0181589F4F0E94CA0681E0809300018E
:1045B00046CF1092680460E08DE594E00E948B097C
:1045C0001092020110920101B7CFEF920F931F9347
:1045D000CF93DF93E80134E047FD34E1042E000C73
:1045E000550B57FF03C0519541955109E32E022FFA
:1045F000242FAE010E940323CE01DF91CF911F91A2
:104600000F91EF900895A9E0B0E0E9E0F3E20C9497
:1046100064266A01F22EB02E102FFBE3AF2EA016F7
:1046200008F41BE31F5F012F27E0AE014F5F5F4FD0
:104630000E946224BC018981982F9970913009F4FD
:104640003FC09BE2E1FC04C09E2D9170E0FC3AC0AB
:104650005E2D5071E82FE87083FF46C084E0911111
:1046600001C083E0EF2DE81B8F1508F0E0E0D601D4
:104670008E2F20E2552351F1992329F0D6019C93E6
:10468000C60101966C0196012D5F3F4FE2FE24C0EA
:104690008EE4D6018C9391E411969C931197129617
:1046A0008C93D9018E2F90E281111BC0E20FF32F62
:1046B000F11D10828EEF9FEF2996ECE00C9480267E
:1046C0009DE2C6CF90E2C4CF2D9381508111FCCFE3
:1046D000CE0ED11CE0E0D0CF8EE6D6018C9391E6D1
:1046E000DBCF9D938150E0CF482F447082FF3DC0C7
:1046F00084E0911101C083E08F1510F4EF2DE81BC9
:10470000D6018E2F20E2552309F1992329F0D601F5
:104710009C93C60101966C0196012D5F3F4FE2FE0E
:104720001BC089E4D6018C938EE411968C9311976B
:1047300086E412968C93D9018E2F90E2882309F497
:10474000B5CF9D938150FACF2D9381508111FCCF2D
:10475000CE0ED11CE0E0D9CF89E6D6018C938EE64F
:1047600011968C93119786E6E4CF9B0177FF02C0E8
:1047700030E020E0A1E0B0E0911102C0B0E0A0E0A4
:10478000F9013196AE0FBF1F8B2C912CBB2009F481
:1047900061C05401EFEFAE1ABE0AAA0DBB1DFA1696
:1047A0001B0619F014F04F2D4A1B511188C0E3FC71
:1047B00059C07601A42FB0E2A1114FC0C40ED11C84
:1047C000992309F45BC040E0D6011196F60190836D
:1047D0006D01552309F448C0012F060F9A81582F07
:1047E000507184FF03C0913309F4015010160CF08E
:1047F00047C0093008F008E0EEE2FE2E5B01A01A87
:10480000B10885019194819491082F3F320729F4D2
:10481000D601FC92F60131966F016217730794F18D
:10482000021713077CF5DB01A21BB30BAA24A39488
:10483000B12CAC0EBD1EAA0DBB1D11968C91215042
:104840003109D601119628153905F4F0F601808357
:104850006D01DBCFB12CA12CA0CFF701B1937F016B
:10486000A150AACF9111B0CFD601942F50E302C02E
:104870005D9391509111FCCFC40ED11C40E0ACCFA0
:1048800001E0BACF80E3DBCF6217730731F49633D0
:1048900088F4953311F4552369F0F6018083FD0106
:1048A000842F90E2811108C0A40FB11D1C9290E0EA
:1048B00080E002CF81E3F1CF91938150F3CF91114A
:1048C00083CF8ACF283008F027E03327DA01990F09
:1048D000311D87FD916000966105710539F43260E4
:1048E0002E5F3D9330E32A95E1F708959F3F30F026
:1048F00080387105610509F03C5F3C5F3D93913064
:1049000008F08068911DDF93CF931F930F93FF9260
:10491000EF92192F987F9695E92F96959695E90F26
:10492000FF27EE53FF4F99273327EE24FF24A701DB
:10493000E70105900894079428F4360FE71EF81E47
:10494000491F511D660F771F881F991F0694A1F7F5
:104950000590079428F4E70EF81E491F561FC11D45
:10496000770F881F991F661F0694A1F7059007947B
:1049700028F4F80E491F561FC71FD11D880F991F15
:10498000661F771F0694A1F70590079420F4490F3E
:10499000561FC71FD81F990F661F771F881F0694C1
:1049A000A9F784911095177041F0D695C795579542
:1049B0004795F794E7941A95C1F7E8E6F0E0689414
:1049C0001590159135916591959105907FE27395BC
:1049D000E118F10A430B560BC90BD009C0F7E10CE3
:1049E000F11E431F561FC91FD01D7EF4703311F4F2
:1049F0008A95E6CFE894015030F0080F0AF40027BA
:104A0000021708F4202F2395022F7A3328F079E338
:104A10007D932A95E9F710C07D932A9589F606942F
:104A200097956795379517951794E118F10A430BF9
:104A3000560BC90BD00998F023957E9173957A3364
:104A400008F070E37C932013B8F77E9170617D933A
:104A500030F0839571E37D9370E32A95E1F711249B
:104A6000EF90FF900F911F91CF91DF91992787FDD4
:104A7000909508950E947C2508F481E00895E894BB
:104A800009C097FB3EF490958095709561957F4F96
:104A90008F4F9F4F9923A9F0F92F96E9BB27939544
:104AA000F695879577956795B795F111F8CFFAF454
:104AB000BB0F11F460FF1BC06F5F7F4F8F4F9F4F85
:104AC00016C0882311F096E911C0772321F09EE8E3
:104AD000872F762F05C0662371F096E8862F70E049
:104AE00060E02AF09A95660F771F881FDAF7880F23
:104AF0009695879597F90895990F0008550FAA0B79
:104B0000E0E8FEEF16161706E807F907C0F01216E0
:104B10001306E407F50798F0621B730B840B950BE3
:104B200039F40A2661F0232B242B252B21F4089538
:104B30000A2609F4A140A6958FEF811D811D0895D5
:104B40000E94B3250C9424260E94162638F00E9459
:104B50001D2620F0952311F00C940D260C9413269D
:104B600011240C9458260E94352670F3959FC1F3AA
:104B7000950F50E0551F629FF001729FBB27F00D0B
:104B8000B11D639FAA27F00DB11DAA1F649F662760
:104B9000B00DA11D661F829F2227B00DA11D621FAF
:104BA000739FB00DA11D621F839FA00D611D221F69
:104BB000749F3327A00D611D231F849F600D211D4D
:104BC000822F762F6A2F11249F5750409AF0F1F0D0
:104BD00088234AF0EE0FFF1FBB1F661F771F881F39
:104BE00091505040A9F79E3F510580F00C940D263E
:104BF0000C9458265F3FE4F3983ED4F3869577955E
:104C00006795B795F795E7959F5FC1F7FE2B880FDE
:104C1000911D9695879597F9089597F99F6780E874
:104C200070E060E008959FEF80EC089500240A94FE
:104C30001616170618060906089500240A94121677
:104C40001306140605060895092E0394000C11F4AA
:104C5000882352F0BB0F40F4BF2B11F460FF04C057
:104C60006F5F7F4F8F4F9F4F089557FD9058440FB0
:104C7000551F59F05F3F71F04795880F97FB991FBB
:104C800061F09F3F79F08795089512161306140678
:104C9000551FF2CF4695F1DF08C016161706180605
:104CA000991FF1CF86957105610508940895E894E0
:104CB000BB2766277727CB0197F908952F923F925C
:104CC0004F925F926F927F928F929F92AF92BF921C
:104CD000CF92DF92EF92FF920F931F93CF93DF93C8
:104CE000CDB7DEB7CA1BDB0B0FB6F894DEBF0FBE25
:104CF000CDBF09942A88398848885F846E847D8472
:104D00008C849B84AA84B984C884DF80EE80FD8073
:104D10000C811B81AA81B981CE0FD11D0FB6F894E9
:104D2000DEBF0FBECDBFED010895A29FB001B39FBE
:104D3000C001A39F700D811D1124911DB29F700DA4
:104D4000811D1124911D08955058BB27AA270E9448
:104D5000BC260C9424260E94162638F00E941D269C
:104D600020F039F49F3F19F426F40C9413260EF426
:104D7000E095E7FB0C940D26E92F0E94352658F3A9
:104D8000BA17620773078407950720F079F4A6F530
:104D90000C9457260EF4E0950B2EBA2FA02D0B0184
:104DA000B90190010C01CA01A0011124FF27591B70
:104DB00099F0593F50F4503E68F11A16F040A22F76
:104DC000232F342F4427585FF3CF469537952795E7
:104DD000A795F0405395C9F77EF41F16BA0B620BE6
:104DE000730B840BBAF09150A1F0FF0FBB1F661F2D
:104DF000771F881FC2F70EC0BA0F621F731F841F70
:104E000048F4879577956795B795F7959E3F08F095
:104E1000B0CF9395880F08F09927EE0F9795879557
:104E200008950E9425270C9424260E941D2658F0E0
:104E30000E94162640F029F45F3F29F00C940D26BD
:104E400051110C9458260C9413260E94352668F3B1
:104E50009923B1F3552391F3951B550BBB27AA2733
:104E600062177307840738F09F5F5F4F220F331F6D
:104E7000441FAA1FA9F335D00E2E3AF0E0E832D035
:104E800091505040E695001CCAF72BD0FE2F29D038
:104E9000660F771F881FBB1F261737074807AB070A
:104EA000B0E809F0BB0B802DBF01FF2793585F4F7F
:104EB0003AF09E3F510578F00C940D260C9458263C
:104EC0005F3FE4F3983ED4F3869577956795B79561
:104ED000F7959F5FC9F7880F911D9695879597F96C
:104EE0000895E1E0660F771F881FBB1F62177307E5
:104EF0008407BA0720F0621B730B840BBA0BEE1FFA
:104F000088F7E09508950E943D2688F09F5798F015
:104F1000B92F9927B751B0F0E1F0660F771F881FBE
:104F2000991F1AF0BA95C9F714C0B13091F00E94D8
:104F30005726B1E008950C945726672F782F8827BD
:104F4000B85F39F0B93FCCF3869577956795B395FF
:104F5000D9F73EF490958095709561957F4F8F4F6E
:104F60009F4F089597FB16F40E94F6270C94B927DB
:104F7000E894F92F96EBFF2381F01216130614061E
:104F8000440B9395F695879577956795579540408F
:104F9000FF23B9F71BC099270895882351F498502F
:104FA000D2F7872B762F652F542F432F322F20E0F7
:104FB000B1F3121613061406440B88233AF09A959F
:104FC000440F551F661F771F881FCAF755234AF4E1
:104FD000440F551F11F460FF04C06F5F7F4F8F4F68
:104FE0009F4F880F9695879597F90895909580958E
:104FF0007095609550954095309521953F4F4F4F56
:105000005F4F6F4F7F4F8F4F9F4F08950E947C25BA
:1050100008F48FEF0895AA1BBB1B51E107C0AA1F1C
:10502000BB1FA617B70710F0A61BB70B881F991F49
:105030005A95A9F780959095BC01CD010895A1E2FC
:105040001A2EAA1BBB1BFD010DC0AA1FBB1FEE1F02
:10505000FF1FA217B307E407F50720F0A21BB30B4D
:10506000E40BF50B661F771F881F991F1A9469F7C9
:1050700060957095809590959B01AC01BD01CF0125
:105080000895DF93CF931F930F939A9DF02D219F47
:10509000F00D8B9DF00D8A9DE02DF10D039FF00D1D
:1050A000029FE00DF11D4E9DE00DF11D5E9DF00D86
:1050B0004F9DF00D7F936F93BF92AF925F934F938D
:1050C000D5010E9495268B01AC01D7010E9495263F
:1050D000EB01E80FF91FD6010E9490282F913F9114
:1050E000D6010E949526C60FD71FE81FF91FAF9162
:1050F000BF910E9490282F913F910E949526C60F44
:10510000D71FE81FF91FD6010E949526E60FF71F4B
:105110009801BE01CF010F911F91CF91DF910895AA
:105120000E949526460F571FC81FD91F08F43196B5
:10513000089597FB57FF0C94A9289F938F930E9483
:10514000A9286E1B7F0BAF91BF918A0B9B0B089513
:10515000E894DF93CF93FC01DB010E9495267F93B7
:105160006F93E9019A01AC01BF93AF933F932F93E3
:10517000DF010E94952626F46C1B7D0B820B930B9E
:105180009E01EB01FC010E949028AF91BF912F91ED
:105190003F910E949028BE01CF01F9012F913F91CC
:1051A000CF91DF910895689401C0E894F92FF12B15
:1051B00012F00C940729A0E0B0E0E1EEF8E20C94C4
:1051C0006426092E059422F40E946329112392F487
:1051D000F0E80F26FFEFE094F09400951095B0945E
:1051E000C094D094A194BF0ACF0ADF0AEF0AFF0A45
:1051F0000F0B1F0B0E94122907FC0E946329CDB7D9
:10520000DEB7ECE00C948026689401C0E8948F929D
:105210009F92CF93DF930E941229DF91CF919F90AD
:105220008F90089588249924F401E401B0E49F93B9
:10523000AA279A158B049C04ED05FE05CF05D0071F
:10524000A10798F4AD2FDC2FCF2FFE2FE92D982C3E
:10525000892E982F872F762F652F542F432F322F8B
:105260002227B85031F7BF9127C01B2EBF91BB2713
:10527000220F331F441F551F661F771F881F991F5A
:10528000881C991CEE1FFF1FCC1FDD1FAA1FBB1F10
:105290008A149B04EC05FD05CE05DF05A007B107C8
:1052A00048F08A189B08EC09FD09CE09DF09A00B1C
:1052B000B10B21601A94E1F62EF49401AF01BE0106
:1052C000CD01000C0895609570958095909530956E
:1052D0004095509521953F4F4F4F5F4F6F4F7F4FF8
:1052E0008F4F9F4F0895002E083090F0982F872FF2
:1052F000762F652F542F432F322F22270850F4CFBB
:10530000220F331F441F551F661F771F881F991FC9
:105310000A95B2F7002D089597FD1094002E0830DD
:1053200098F00850232F342F452F562F672F782FB2
:10533000892F912DF4CF159497958795779567953B
:1053400057954795379527950A95AAF71124002D6B
:1053500008952A0D3B1D4C1D5D1D6E1D7F1D801F78
:10536000911F08952A193B094C095D096E097F09AF
:10537000800B910B0895EE0FFF1F0590F491E02D27
:1053800009940F931F93CF93DF938230910510F40C
:1053900082E090E0E0916B04F0916C0430E020E05A
:1053A000B0E0A0E0309799F42115310509F44AC026
:1053B000281B390B24303105D8F58A819B81611572
:1053C000710589F1FB0193838283FE0111C0408145
:1053D00051810281138148175907E0F04817590796
:1053E00099F4109761F012960C93129713961C93F0
:1053F0003296CF01DF91CF911F910F9108950093C5
:105400006B0410936C04F4CF2115310551F0421751
:10541000530738F0A901DB019A01BD01DF01F80152
:10542000C1CFEF01F9CF90936C0480936B04CDCF83
:10543000FE01E20FF31F81939193225031093983CA
:105440002883D7CF2091690430916A04232B41F43B
:10545000209105013091060130936A04209369047C
:1054600020910301309104012115310541F42DB73C
:105470003EB74091070150910801241B350BE09184
:105480006904F0916A04E217F307A0F42E1B3F0BA6
:105490002817390778F0AC014E5F5F4F24173507A6
:1054A00048F04E0F5F1F50936A0440936904819344
:1054B00091939FCFF0E0E0E09CCFCF93DF930097F4
:1054C000E9F0FC01329713821282A0916B04B09133
:1054D0006C04ED0130E020E01097A1F420813181CF
:1054E000820F931F2091690430916A0428173907AD
:1054F00009F061C0F0936A04E0936904DF91CF91F1
:105500000895EA01CE17DF07E8F54A815B819E0125
:1055100041155105B1F7E901FB83EA83499159919E
:10552000C40FD51FEC17FD0761F4808191810296AD
:10553000840F951FE90199838883828193819B83DE
:105540008A83F0E0E0E012968D919C91139700978A
:10555000B9F52D913C911197CD010296820F931FC1
:105560002091690430916A042817390739F6309779
:1055700051F510926C0410926B04B0936A04A093DE
:105580006904BCCFD383C28340815181840F951FAE
:10559000C817D90761F44E5F5F4F88819981480F22
:1055A000591F518340838A819B8193838283211574
:1055B000310509F0B0CFF0936C04E0936B049ECFFB
:1055C000FD01DC01C0CF13821282D7CFB0E0A0E092
:1055D000ECEEFAE20C9460268C01009751F4CB01BA
:1055E0000E94C1298C01C801CDB7DEB7E0E10C945F
:1055F0007C26FC01E60FF71F9C0122503109E217BF
:10560000F30708F49DC0D901CD91DC911197C6171D
:10561000D70798F0C530D10530F3CE01049786172F
:10562000970708F3C61BD70B2297C193D1936D93AD
:105630007C93CF010E945D2AD6CF5B01AC1ABD0AD4
:105640004C018C0E9D1EA0916B04B0916C04512CEA
:10565000412CF12CE12C109731F580916904909147
:105660006A048815990509F05CC04616570608F0CB
:1056700058C08091030190910401009741F48DB7C7
:105680009EB74091070150910801841B950BE817C4
:10569000F90708F055C0F0936A04E0936904F90132
:1056A00071836083A0CF8D919C91119712966C901D
:1056B000129713967C901397A815B90559F56C01AC
:1056C00042E0C40ED11CCA14DB0420F1AC014A191B
:1056D0005B09DA011296159780F06282738251831A
:1056E0004083D9016D937C93E114F10471F0D701EB
:1056F0001396FC93EE93129776CF22968C0F9D1FF4
:10570000F90191838083F301EFCFF0936C04E09370
:105710006B0469CF4816590608F42C017D01D301AA
:105720009ACFCB010E94C1297C01009749F0AE01BC
:10573000B8010E94A32BC8010E945D2A870153CFA4
:1057400010E000E050CFFB01DC0102C001900D929F
:1057500041505040D8F70895FB01DC018D91019034
:1057600080190110D9F3990B0895FB01DC01019018
:105770000D920020E1F70895F894FFCF0101000099
:10578000006D04800000004000140054000100007F
:1057900000020000000300000005000000090000F6
:1057A00000110000000100000002000000030000E2
:1057B000000500000009000000120000000000C009
:1057C000BF0000803F000000C000008040000000DB
:1057D000C00000000046079D06D30693070407E2B9
:1057E00006F606000000005C092F09A00918092828
:1057F0000947051909000000003B0F9D06A009B3E9
:10580000072F2F22225C5C6208660C6E0A720D74F0
:1058100009005C7530303030006E756C6C0074724D
:1058200075650066616C73650068756D69007072FE
:105830006573004E6170616B612073656E7A6F7283
:105840006A61203321004E6170616B612073656E67
:105850007A6F726A61203221004E6170616B612043
:1058600073656E7A6F726A61203121004E617061DA
:105870006B612073656E7A6F726A61203421006FEC
:10588000626A5F74656D70004E6170616B61207358
:10589000656E7A6F726A6120352100543A200020CB
:1058A0004300483A20002025524800503A2000206A
:1058B0006850610074656D70657261747572650021
:1058C00068756D6964697479007072657373757257
:0658D00065000D0A000056
:107E0000112484B714BE81FFF0D085E080938100F7
:107E100082E08093C00088E18093C10086E0809377
:107E2000C20080E18093C4008EE0C9D0259A86E02C
:107E300020E33CEF91E0309385002093840096BBD3
:107E4000B09BFECF1D9AA8958150A9F7CC24DD24C4
:107E500088248394B5E0AB2EA1E19A2EF3E0BF2EE7
:107E6000A2D0813461F49FD0082FAFD0023811F036
:107E7000013811F484E001C083E08DD089C08234E0
:107E800011F484E103C0853419F485E0A6D080C0E4
:107E9000853579F488D0E82EFF2485D0082F10E0AE
:107EA000102F00270E291F29000F111F8ED06801E7
:107EB0006FC0863521F484E090D080E0DECF843638
:107EC00009F040C070D06FD0082F6DD080E0C81688
:107ED00080E7D80618F4F601B7BEE895C0E0D1E017
:107EE00062D089930C17E1F7F0E0CF16F0E7DF06D8
:107EF00018F0F601B7BEE89568D007B600FCFDCFD4
:107F0000A601A0E0B1E02C9130E011968C91119780
:107F100090E0982F8827822B932B1296FA010C0160
:107F200087BEE89511244E5F5F4FF1E0A038BF0790
:107F300051F7F601A7BEE89507B600FCFDCF97BE46
:107F4000E89526C08437B1F42ED02DD0F82E2BD052
:107F50003CD0F601EF2C8F010F5F1F4F84911BD097
:107F6000EA94F801C1F70894C11CD11CFA94CF0C13
:107F7000D11C0EC0853739F428D08EE10CD085E9AC
:107F80000AD08FE07ACF813511F488E018D01DD067
:107F900080E101D065CF982F8091C00085FFFCCF94
:107FA0009093C60008958091C00087FFFCCF809118
:107FB000C00084FD01C0A8958091C6000895E0E648
:107FC000F0E098E1908380830895EDDF803219F02E
:107FD00088E0F5DFFFCF84E1DECF1F93182FE3DFCA
:107FE0001150E9F7F2DF1F91089580E0E8DFEE27F6
:047FF000FF270994CA
:027FFE00040479
:00000001FF
